:100979002321323030454655002324323030454654
:02098900550017
:10094E00AF8475840F758A83E4F58475C04475CFC2
:05095E00E4C2C38F8418
:010963002271
:0608E2008F27AD27AF26B1
:0208E8008D1E63
:1008EA001208C0EFC454F0F51FAF1E1208C0EF255E
:0408FA001FF51FFFC8
:0108FE0022D7
:100899008F828E83D3E5829DE5839C501943B701EE
:1008A900758F03E4F0F58F53B7FE2582F582740442
:0608B9003583F58380DEAB
:0108BF002216
:02061400A90734
:1006160020C3FD20C5FAC2C4D2C5E4FFFC30C3FD29
:1006260030C3FDE5C154F8FA64086003BA1011E559
:100636001DBF01044401800254FEF5C27C01807C8A
:10064600BA180B851CC27C02C2C4C2C5806EBA2011
:10065600028038EA64287030B9010CBC02028015A9
:10066600EC6404701F8019BC02088BC27C03C2C5EF
:100676008012BC03088DC27C04C2C58007BC04047A
:10068600D2C57F01C2C48034BA300AD2C4D2C57C76
:1006960009E4FF8027BA3802801EBA4006C2C2C2E9
:1006A600C58019BA48028010BA50028003BA5808A9
:1006B600D2C47C08AEC28004D2C4D2C5C2C3EC6424
:0806C600086003020626AF06DE
:0106CE002209
:10099C00AE05AD078E1C8B1DE4FB7F0112061422E5
:10098B00AE03AB05AD078E1C751DA07F02120614BE
:01099B002239
:06027A008B3D8A3E893F26
:100280007547FF75480975497975440175450075CD
:100290004600E4F543F542F541F540E47F50FEFDAC
:1002A000FCAB43AA42A941A840C31207275036AF6E
:1002B000437BA0E4FD12099CAB440546E546AA45F4
:1002C0007002054514F9EF120715E4FAF9F8E54351
:1002D0002401F543EA3542F542E93541F541E83577
:1002E00040F54080B6AB47AA48A9491206CFFF9017
:1002F0000000E06F70629000011206E8FF900001BC
:10030000E06F70549000021206E8FF900002E06F68
:1003100070469000031206E8FF900003E06F70380B
:100320009000041206E8FF900004E06F702A90002D
:10033000051206E8FF900005E0B5071C90000612C4
:1003400006E8FF900006E0B5070E9000071206E8E9
:10035000FF900007E06F60037F0022AB3DAA3EA93B
:100360003F1206CFFF900011E06F702A900001123B
:1003700006E8FF900012E0B5071C9000021206E8A4
:10038000FF900013E0B5070E9000031206E8FF90FF
:100390000014E06F60037F0022900009E0F55BA38A
:1003A000E0F55DA3E0F55E900019E0F557A3E0F5F8
:0703B00059A3E0F55A7F019B
:0103B7002223
:0D08FF008F0DAF18AE171209648E178F18F9
:02090C00AC0637
:0D090E00AB07AF04AD07AF03AB5812099C57
:01091B0022B9
:0E09BB00E55CC3955B500605580558055C22A7
:100964000FBF00010ED3EF955EEE955D40061209B0
:05097400BBE4FEFF22C0
:0403B8008E088F0913
:1003BC00E4F50DF50EF513F514F515F516F517F521
:1003CC0018855917855A18855758F50EF50D755C13
:1003DC0001E4F512E50D643A6016AF18AE17120978
:1003EC000C8F0DAF18AE171209648E178F1880E49E
:1003FC000514E51470020513AF18AE1712090C1290
:10040C0008FF8F0EAD0EAF0D1208E88F108510127D
:10041C001209011208FF8F0EAD0EAF0D1208E87510
:10042C0015008F16EF2512F512E516751600F51549
:10043C001209011208FF8F0EAD0EAF0D1208E8EF76
:10044C00421685150A85160BE5162512F5121209AA
:10045C00011208FF8F0EAD0EAF0D1208E88F0FE5DD
:10046C000F2512F512E50F705CF50CE50CC3951019
:10047C0050531209011208FF8F0EAD0EAF0D12086A
:10048C00E88F11E5112512F512C3E50B9509E50A64
:10049C009508402DAE0AAF0BBEFB06BFFE0343B161
:1004AC003043B701758F01850B82850A83E511F006
:1004BC00E4F58F53B7FE75B111050BE50B70020512
:1004CC000A050C80A61209011208FF8F0EAD0EAFA3
:1004DC000D1208E88F11E5112512700AE50F640161
:0604EC0060030203DD22A3
:0104F20022E7
:0604F3008B4A8A4B894C84
:1004F9007554FF7555097556827551017552007508
:100509005350E4F550F54FF54EF54DE47F2BFEFDC4
:10051900FCAB50AA4FA94EA84DC31207275035AFBF
:1005290050E4FBFD12098BAB510553E553AA5270F8
:1005390002055214F9EF120715E4FAF9F8E5502407
:1005490001F550EA354FF54FE9354EF54EE8354D91
:10055900F54D80B7AB54AA55A9561206CFFF9000A6
:1005690050E06F70629000011206E8FF900051E0C0
:100579006F70549000021206E8FF900052E06F700D
:10058900469000031206E8FF900053E06F70389020
:1005990000041206E8FF900054E06F702A900005ED
:1005A9001206E8FF900055E0B5071C9000061206F8
:1005B900E8FF900056E0B5070E9000071206E8FF25
:1005C900900057E06F60037F0022AB4AAA4BA94C09
:1005D9001206CFFF90005FE06F702A9000011206AB
:1005E900E8FF900060E0B5071C9000021206E8FFE2
:1005F900900061E0B5070E9000031206E8FF900035
:0A06090062E06F60037F00227F01B2
:0106130022C4
:10085000E48F34F533F532F531AE33AD32AC317867
:10086000081207508F348E338D328C317835120751
:010870006324
:080871008F628E618D608C5FC7
:10087900AA07780812073DA907AF62AE61AD60AC5F
:0F0889005F781012073DAB07AF02AD0112098B6C
:01089800223D
:0400A6008E218F22F6
:1000AA00E4F526F527F534F533F532F531F538F56B
:1000BA0037F536F535F53CF53BF53AF53975382B14
:1000CA00F537F536F535F527F526F52CE4F52BE564
:1000DA0026643A600712086C8F2680F3E53C2401F7
:1000EA00F53CE4353BF53BE4353AF53AE43539F588
:1000FA003912086C8F2612086C1208E28F2985299A
:10010A002B12086C8F2612086C1208E2E48F30F565
:10011A002FF52EF52DEF252BF52BAE2FAD2EAC2D71
:10012A0078081207508F308E2F8D2E8C2D12086C66
:10013A008F2612086C1208E2E5304FF530E52FF5EC
:10014A002FE52EF52EE52DF52D852F23853024E577
:10015A0030252BF52B12086C8F2612086C1208E238
:10016A008F28E528252BF52BE5286404703B120817
:10017A006C8F2612086C1208E21208508F26120899
:10018A006C1208E2E5344FF534E533F533E532F520
:10019A0032E531F531AF34AE33AD32FC78101207A7
:1001AA00508F348E338D328C31E5286402703B12C5
:1001BA00086C8F2612086C1208E21208508F261259
:1001CA00086C1208E2E5344FF534E533F533E532CD
:1001DA00F532E531F531AF34AE33AD32FC78041285
:1001EA0007508F348E338D328C31E5342524F52433
:1001FA00E5333523F523E5287058F525E525C3951C
:10020A0029504F12086C8F2612086C1208E28F2AA6
:10021A00E52A252BF52BC3E5249522E523952140D4
:10022A002DAE23AF24BEFB06BFFE0343B13043B756
:10023A0001758F01852482852383E52AF0E4F58FF1
:10024A0053B7FE75B1110524E5247002052305256F
:10025A0080AA12086C8F2612086C1208E28F2AE50F
:0F026A002A252B700AE528640160030200D622C2
:010279002262
:0500060032323245001A
:1009360090007BE584F075840F75E107D2FA75E3C4
:07094600C075A4FFE0F58479
:01094D002287
:0300160002094E8E
:0F09AC00120936E5B05404FFEF7002D322C322C4
:10078300C200C201C20275FFDE75FFAD1209AC9251
:100793000030005E1200167BFF7A00790612027A9F
:1007A300EF24FF92013001147D007CB07F007E4076
:1007B3001208997F007E401203B880237BFF7A00E2
:1007C30079061204F3EF24FF92023002127D007CBB
:1007D300B07F007E401208997F007E401200A6E49D
:1007E300FFFE0FBF00010EBE27F8BF10F5E4F5842E
:0507F300F5C002000E3C
:04000E00024000228A
:01FBFE00FE08
:0300000002091CD6
:03000300025003A5
:03000B000250069A
:030013000250098F
:03001B0002500C84
:0300230002500F79
:03002B000250126E
:0300330002501563
:03003B0002501858
:0300430002501B4D
:03004B0002501E42
:0300530002502137
:03005B000250242C
:0300630002502721
:03006B0002502A16
:0300730002502D0B
:03007B0002503000
:03008300025033F5
:03008B00025036EA
:03009300025039DF
:03009B0002503CD4
:0300A30002503FC9
:10091C00787FE4F6D8FD9000007F007E20E4F0A301
:0A092C00DFFCDEFA7581620207832A
:10080000E590540C23C0E0740AC0E0C082C08302AB
:100810000A00E590540C23C0E0740AC0E0C082C016
:1008200083020A08E590540C23C0E0740AC0E0C0BB
:1008300082C083020A10E590540C23C0E0740AC001
:08084000E0C082C083020A1827
:040A00005390F322FA
:070A080043900C5390F7220C
:070A100043900C5390FB2200
:040A180043900C22D9
:07084800EFC403900A0073E6
:1006CF00BB010689828A83E0225002E722BBFE0229
:0906DF00E32289828A83E493225C
:1006E800BB010CE58229F582E5833AF583E02250C7
:1006F80006E92582F8E622BBFE06E92582F8E22211
:0D070800E58229F582E5833AF583E493222A
:10071500BB010689828A83F0225002F722BBFE01C3
:02072500F322BD
:10072700EB9FF5F0EA9E42F0E99D42F0EC6480C849
:0607370064809845F022E9
:10073D00E8600FECC313FCED13FDEE13FEEF13FF9A
:03074D00D8F122BE
:10075000E8600FEFC333FFEE33FEED33FDEC33FC07
:03076000D8F122AB
:100763007401FF3395E0FEFDFC080808E6CF2FF681
:1007730018E6CE3EF618E6CD3DF618E6CC3CF6225A
:1008C000EF7E0024D0B40A00401624F9B40A004098
:1008D0000CB41000400A24E0B41000400374FFFE82
:0208E000FF22F5
:00000001FF
